:1000000012C02CC02BC02AC029C028C027C026C0BF
:1000100025C024C023C022C021C020C01FC01EC0D4
:100020001DC01CC01BC011241FBECFE5D4E0DEBF25
:10003000CDBF10E0A0E6B0E0E4E9F0E002C005903A
:100040000D92A036B107D9F710E0A0E6B0E001C0EC
:100050001D92A036B107E1F70ED01BC0D1CF9C0195
:1000600006C080EF90E00197F1F721503040211554
:100070003105B9F70895CFE5D4E0DEBFCDBFA59A2D
:10008000AD9884EF91E0EBDFAD9A84EF91E0E7DF8C
:04009000F7CFFFCFD8
:00000001FF
